:1000000000308A009D2A00000A108A100A11820717
:1000100028340C34013406340A108A100A1182077D
:10002000413454342B3443344D3447344C343D3410
:1000300031340D3400340A108A100A1182070C344E
:100040004E3465346E34693420346E346F34763413
:100050006134203453344D34533420347A34703482
:10006000723461347634613400340A108A100A1113
:10007000820700340A108A100A1182075A34613448
:1000800073346C34653474346534203453344D34F3
:10009000533420346E34613420346334693473341F
:1000A0006C346F3400340A108A100A11820720342D
:1000B000203420342034373433343634203436344A
:1000C00035343534203432343534303400340A1089
:1000D0008A100A1182070C345034723469346A343D
:1000E000613474346134203453344D345334203407
:1000F00073342034743465347834743465346D3436
:1001000000340A108A100A1182070C3420344F344C
:10011000643473347434723461346E3465346E34E0
:1001200069342034763465346C346B347934633418
:10013000683400340A108A100A11820720342034EF
:100140002034203420342034203470346934733423
:100150006D3465346E3400340A108A100A11820737
:100160000C3400340A108A100A11820720345A34E1
:10017000613470346E34753474346F3420347A34AE
:100180006134723469347A3465346E3469342034BD
:10019000313400340A108A100A1182072034563490
:1001A000793470346E34753474346F3420347A3466
:1001B0006134723469347A3465346E34693420348D
:1001C000313400340A108A100A1182072034203496
:1001D0005034723465346A34693420346834653498
:1001E0007A346B3479342034643465346E34213499
:1001F0000034000000000A148A100A11023E03189D
:100200008A0A82002034203420342034503472345E
:1002100069346B3461347A3420346E34653462343A
:1002200079346C3400340A148A100A11820720349D
:100230002034203420342034203472346F347A3423
:1002400065347A346E3461346E3400345230840054
:10025000000803193B290530F800BF30F70064009F
:10026000F70B2F29F80B2D29F930F700F70B36295A
:100270006400800B2B2900340708F039D900580896
:100280000F3959048700061483160610640098304D
:10029000F700F70B492900000000831206108316AF
:1002A0000610831200340430D802031C6B29583026
:1002B0008400F83080050310800C800C800C00084E
:1002C00003196B290A30F700F70B642900000000BE
:1002D0006400800B62298A110A128329D608031D43
:1002E0007329861074298614831686108312D70EFC
:1002F0005708D8003C21D70E5708D8003C2164008D
:10030000C730D800532900341430D2002621F030F1
:1003100083168705831286108316861083120610B3
:10032000831606108312D0015008023C031CA0293A
:100330000230D20026210330D8003C21D00A942973
:1003400064003C30F700F70BA329000000000230E6
:10035000D8003C2164003C30F700F70BAD290000C9
:100360000000D0015008023C031CC22950080420A0
:10037000D100D6015108D7006E210230D2002621CB
:10038000D00AB22900342013200883168700831274
:1003900007130830F800000000000000F817DF29FC
:1003A000F813D10C03180717031C07137817DF295C
:1003B0007813F80BD129000000000000071749301E
:1003C0008400840BE129000000000000F81BD02904
:1003D000781BD8298A110A12242B0830F700A0179D
:1003E0002008831687008312871FF8298316F329B4
:1003F000D001F717092AF713092A0310871B0314E2
:10040000D00C7717092A7713F70BFD295008F8004D
:10041000162A4930F71B1430F800F80B0D2A00009B
:100420000000F71BFB29771B032AFD29003401304C
:100430005302FC3E0318292A043E342AD401292AF7
:100440004030D400292A1430D400292A5430D40052
:10045000292A01305202D40754088038D500D60129
:100460005508D7006E2100340A108A140A11820739
:100470001E2A202A232A262A51080C3A03194A2A1E
:10048000063A0319522A073A0319582A053A03195A
:100490005D2A622AD6010130D7006E210230D200D7
:1004A00026216E2A0130D2000230D30017226E2A94
:1004B0000130D200D30017226E2AD6011030D700A7
:1004C0006E216E2A51081F3C031C682A0730D10593
:1004D0000130D6005108D7006E216E2A00348316F1
:1004E0000611831206110830F80000000000000019
:1004F000F817892AF813D10C03180615031C0611E6
:100500007817892A7813F80B7B2A00000000000076
:1005100006150930F7008401840B8C2AF70B8B2A0F
:10052000F0308400840B922A00000000F81B7A2A25
:10053000781B822A8A110A12142D84011F30830528
:1005400020132008831687008312071783160611CD
:100550008312061583161F149F141F159F11073051
:100560009C00FF308312A00083161F149F141F15D8
:100570009F1183121F109412A01220088316870067
:10058000831220162008831687008312A0112008EA
:100590008316870001308312940000308316940084
:1005A0000108C73908388100831290010030F80033
:1005B000920000308316920007309C00050864000A
:1005C0000E30F700F70BE22A000000001C0883122F
:1005D0000D1383169D010F30F70007308312810140
:1005E000813084000008F03907388000640000087A
:1005F000F739F719F03977048000842164008316F5
:100600000512831205129630D20026218316051298
:10061000831205169630D200262183160512831206
:1006200005129630D2002621831605128312051674
:100630009630D2002621D00150080C200038031932
:10064000252BD00AD100C3291C2BED2178080A3CA8
:10065000031D252BED217808A100ED217808A200CB
:10066000ED2178080A3C031D302B831605128312F6
:10067000051621084F3C031D842B22084B3C031D0B
:10068000842B0130D200D3001722D00150081B2048
:10069000003803194F2BD00AD1003C22462B0130E1
:1006A000D2000230D3001722D00150083520003884
:1006B00003195E2BD00AD1003C22552B0130D20009
:1006C0000330D3001722D00150083A200038031914
:1006D0006D2BD00AD1003C22642B0130D2000430B3
:1006E000D3001722D00150085320003803197C2B67
:1006F000D00AD1003C22732B1430D000FA30D20043
:100700002621D00B7E2BDF2DC9014908353C031C67
:100710008C2BED21C90A852BED217808A100ED2154
:100720007808A200ED217808A300ED217808A40044
:10073000ED217808A500ED217808A600ED217808C4
:10074000A700ED217808A800A108031DA92B3030CF
:10075000A2003030A102A2022108093C0318B22BEA
:100760000730A1022208093C0318B82B0730A20267
:10077000A10EF030A1052208A104A308031DC22B7D
:100780003030A4003030A302A4022308093C03182F
:10079000CB2B0730A3022408093C0318D12B0730C8
:1007A000A402A30EF030A3052408A304A508031D8A
:1007B000DB2B3030A6003030A502A6022508093C0C
:1007C0000318E42B0730A5022608093C0318EA2B7E
:1007D0000730A602A50EF030A5052608A504A70837
:1007E000031DF42B3030A8003030A702A8022708E0
:1007F000093C0318FD2B0730A7022808093C031801
:10080000032C0730A802A70EF030A7052808A7047C
:100810002308A2002508A3002708A400A701270891
:10082000A600A500CB01C9014908033C031C6B2CA1
:100830000310CE0CCE1721304907840000084E0566
:10084000CC0021304907D00021304907840000083E
:10085000F7004B08F8000319312C0310F70DF80BC3
:100860002D2C5008840077088000CA014B08083CF2
:100870004A020318402C0310CD0CCD13CA0A362CA3
:1008800021304907D00021304907840000084D0479
:10089000D200500884005208800021304907D0005F
:1008A00021304907840000087F39D20050088400B5
:1008B000520880004C08CD00CB0A4B08083C031DB1
:1008C000692CCB0101304907213E84004D0880008E
:1008D000CE01C90A142C21304907840080018421EB
:1008E0000130D200D3001722D00150086720003811
:1008F00003197E2CD00AD1003C22752C0930D2007D
:100900000330D30017222130840000300004031983
:10091000922C0408D0000008D1003C22500884002A
:10092000840A852C83160512831205120430D00028
:10093000FA30D2002621D00B982C83160512831290
:1009400005162108403C0318AB2C21085A3C031C17
:10095000AB2C2030A1072208403C0318B52C2208FC
:100960005A3C031CB52C2030A2072308403C031836
:10097000BF2C23085A3C031CBF2C2030A30724089B
:10098000403C0318C92C24085A3C031CC92C2030B5
:10099000A4070130D200D3001722D00150088120D3
:1009A00000380319D72CD00AD1003C22CE2C0130BC
:1009B000D2000230D3001722D00150089A2000380C
:1009C0000319E62CD00AD1003C22DD2C0930D200DC
:1009D0000430D300172221308400003000040319B2
:1009E000FA2C0408D0000008D1003C2250088400F2
:1009F000840AED2C83160512831205120430D000F0
:100A0000FA30D2002621D00B002D83160512831256
:100A1000051621308400003000040319182D040845
:100A2000D0000008D1006F2A50088400840A0B2DE2
:100A300021087A3C031D2A2D2208613C031D2A2D22
:100A40002308703C031D2A2D2408313C031D2A2D48
:100A50000130CF002108763C031D3C2D2208793C53
:100A6000031D3C2D2308703C031D3C2D2408313C04
:100A7000031D3C2D0230CF002108613C031D4E2D8B
:100A80002208683C031D4E2D23086F3C031D4E2D8C
:100A900024086A3C031D4E2D0330CF004F08013A55
:100AA0000319592D033A0319772D013A0319952D8E
:100AB000AF2D8316851183128511D0015008AC200B
:100AC00000380319672DD00AD1003C225E2D013079
:100AD000D2000230D3001722D0015008B2200038D3
:100AE0000319762DD00AD1003C226D2DD82D831606
:100AF000851183128515D0015008AC2000380319E8
:100B0000852DD00AD1003C227C2D0130D20002304C
:100B1000D3001722D0015008CA2000380319942DA1
:100B2000D00AD1003C228B2DD82DD0015008AC200A
:100B3000003803199F2DD00AD1003C22962D013098
:100B4000D2000230D3001722D0015008E220003832
:100B50000319AE2DD00AD1003C22A52DD82DD001ED
:100B60005008AC2000380319B92DD00AD1003C221E
:100B7000B02D0130D2000230D3001722D00150082E
:100B8000F92000380319C82DD00AD1003C22BF2D0E
:100B90000130D2000330D3001722D00150081321B6
:100BA00000380319D72DD00AD1003C22CE2DD82DE4
:100BB0000430D000FA30D2002621D00BDA2DFE2AE4
:020BC0006300D0
:02400E003A3F37
:00000001FF
